:020000040000FA
:1000000000008A110A12012BF200030E8301F10095
:100010000A088A01F000040883160313E60083121D
:1000200003130B1D17288714810187100B118316EA
:1000300003136608840070088A008301710E830030
:10004000F20E720E0900C422831203138B1783165B
:100050000313D7010C3083160313570203184028EB
:100060005708DA3ED80000300318013ED90058087E
:100070008400831359188317FF308000D70A2A2879
:100080006F2083160313D70118308316031357020A
:1000900003185A285708203ED80000300318013EA4
:1000A000D90058088400831359188317FF30800043
:1000B000D70A44289A208312031388186028F9204D
:1000C0000030831203136D04031D9A200030831245
:1000D00003136E0403195B286F205B2808000B30A4
:1000E00083120313010203186F28091507108316E2
:1000F0000313CE010C30831603134E02031892280B
:100100004E08DA3ECF0000300318013ED0004F0801
:1001100084008313501883170008D7208316031315
:10012000CE0A7A28831203130714071083120313CD
:10013000EE0108000B3083120313010203189A2802
:10014000091DA8280911013083160313CE00AB281E
:1001500083160313CE0183160313CF014830831691
:1001600003134F020318C6284F08203ED00000306A
:100170000318013ED10050088400831351188317DF
:100180000008D72083160313CF0AAE288312031367
:1001900007140710831603134E080319D32883127C
:1001A00003138715871183120313ED0108008316CB
:1001B0000313D200D6010830831603135602031826
:1001C000F828D21FE728831203138716EA28831220
:1001D0000313871283120313871503108316031367
:1001E000D20D83120313871183160313D60ADB285B
:1001F0000800B02283160313CE004E0803192529E8
:100200004E08013A03192A294E08023A03192F29E8
:100210004E08033A031951294E08803A03197329ED
:100220004E08813A031978294E08823A03197C292D
:100230004E08F33A031980294E08F43A0319382A74
:100240004E08F53A03198C2A942A013083120313BD
:10025000ED00942A013083120313EE00942A8316D2
:100260000313CE014830831603134E0203184C29A2
:100270004E08203ECF0000300318013ED000B022CF
:1002800083160313D1004F0884008313501883177B
:1002900051088000CE0A3229013083120313ED0089
:1002A000942A83160313CE010C30831603134E02D7
:1002B00003186E294E08DA3ECF0000300318013EC5
:1002C000D000B02283160313D1004F08840083139B
:1002D0005018831751088000CE0A54290130831228
:1002E0000313EE00942A2030831203138806942A05
:1002F000831203138B13942A831203138B17942AEC
:1003000083160313CE010530831603134E02031820
:10031000942A0930FF004E088A110A12C9238A1153
:100320000A1283160313CF00A03ED000003003183A
:10033000013ED10050088400831351188317000830
:10034000D200840A0008D0008403D101D01BD1035D
:100350005008D2009522831603134F08A03ED00008
:1003600000300318013ED100500884008313511857
:1003700083170008D200840A0008D30084035208BF
:10038000D0009522831603134F08A03ED000003002
:100390000318013ED2000230D0070318D20A5008D9
:1003A00084008313521883170008D300840A0008BE
:1003B000D0008403D201D01BD2035008D300952271
:1003C000831603134F08A03ED00000300318013EEF
:1003D000D2000230D0070318D20A500884008313D9
:1003E000521883170008D300840A0008D40084033D
:1003F0005308D0009522831603134F08A03ED00067
:1004000000300318013ED3000430D0070318D30A8C
:10041000500884008313531883170008D400840AFB
:100420000008D0008403D301D01BD3035008D400AC
:100430009522831603134F08A03ECF000030031807
:10044000013ED0000430CF070318D00A4F088400C3
:100450008313501883170008D300840A0008D400BF
:1004600084035308CF00952283160313CE0A8329F1
:1004700083160313CE010530831603134E020318AF
:10048000942A0930FF004E088A110A12C9238A11E2
:100490000A1283160313CF00A03ED30000300318C6
:1004A000013ED4000630D3070318D40A5308840051
:1004B0008313541883170008D5009522831603135D
:1004C0004F08A03ED30000300318013ED40007308F
:1004D000D3070318D40A53088400831354188317CE
:1004E0000008D5009522831603134F08A03ECF00C5
:1004F00000300318013ED3000830CF070318D30A99
:100500004F0884008313531883170008D4009522E2
:1005100083160313CE0A3B2A831203136D08952218
:10052000831203136E089522080083160313CD006F
:100530008316031386013F308805831603134D0885
:10054000831203138600831203130818A32A881149
:100550008815FF30831603138600C0308804080016
:10056000831203130816831203138818B32A081280
:100570000811060883160313CD0083120313081510
:10058000831603134D080800831203138B018101A6
:100590008B1697019D019401831603138C018D0125
:1005A00083120317870188017830831603138F00A5
:1005B00003308100831203138501860187018801BE
:1005C00089010815881589140915871407108711E2
:1005D00083160317880183160313850183160317F7
:1005E0008901FF3083160313860010308700C33063
:1005F0008800890183120313ED0183120313EE01B6
:100600000800E630FE000330FF0080308A110A1235
:10061000A8238A110A128312031791007F08900001
:10062000E8309200033093008312031710089400FF
:1006300011089500FF309007031C9103140815045E
:100640000319912B0430120794009501950D13089E
:1006500095071408FE001508FF0080308A110A1261
:10066000A8238A110A128312031797007F089600A5
:100670001208FE001308FF0080308A110A12A82316
:100680008A110A1283120317990095007F089800B7
:1006900094000230120794009501950D13089507F8
:1006A0001408FE001508FF0080308A110A12A823E2
:1006B0008A110A128312031795009B007F08940089
:1006C0009A008312031716089A0017089B00FF3040
:1006D0009607031C97031A081B0403198A2B180892
:1006E000FE001908FF0080308A110A1295238A1132
:1006F0000A12831203179A00140884008313151832
:1007000083171A088000980A0319990A940A031992
:10071000950A612B06308312031792070318930A78
:10072000142B8A110A1223280800003A03199C2B63
:10073000803A0319A32B00347E08840083137F18AA
:100740008317000808007F088A007E0882000800DE
:10075000003A0319B02B803A0319BA2BFF01003479
:100760007E08840083137F1883170008FF00840A23
:10077000000808008A110A12A323FD00FE0FFF03E0
:10078000FF0A8A110A12A323FC007D08FF007C08DF
:10079000080083120313E8007F08E900EA0108302B
:1007A000EB0083120313681CD72B6908EA07831236
:1007B00003136808EC0003106C0CE8000310690DCB
:1007C000EC00E900EB0BD12B6A080800013400347F
:0E07D000EE340334E7340034013400340034D6
:02400E00F5209B
:02401000FC3F73
:00000001FF
